:1038000011241FBECFEFD4E0DEBFCDBF11E0A0E09A
:10381000B1E0EEEAFBE302C005900D92A030B107E3
:10382000D9F711E0A0E0B1E001C01D92A238B107C4
:10383000E1F70C943B1C0C941D1C0895982F80916B
:10384000C00085FFFCCF9093C60008958091C00012
:103850008823E4F78091C600992708958DE40E949B
:103860001E1C8BE40E941E1C82E40E941E1C8CE421
:103870000E941E1C0895CFEFD4E0DEBFCDBFE0E074
:10388000F0E004917F01992494BE98E10FB6F8947A
:1038900090936000109260000FBE9092C50080E18E
:1038A0008093C4008091C00082608093C000909398
:1038B000C10086E08093C200EF01192D8091C00005
:1038C00087FF0DC0113031F48091C6008A3A89F12A
:1038D00010E005C08091C6008B3109F411E0CE01E3
:1038E00021968436910500F10F3F41F0002331F01D
:1038F000E0910001F0910101099516C08AE00E9453
:103900001E1C8DE00E941E1C86E50E941E1C80E38A
:103910000E941E1C8EE20E941E1C82E30E941E1C3E
:103920008AE30E941E1C05C080E29EE40197F1F725
:10393000C5CF0E942E1C0E94261C813611F489E5F9
:1039400033C1813471F40E94261CE82EFF24FE2C22
:10395000EE240E94261C9927E82AF92AF694E79477
:10396000F1C0823641F489E50E941E1C80E00E946D
:103970001E1C80E819C1823409F075C00E94261C03
:103980000E94261CD82E0E94261C082FB2E0AB2EC7
:10399000B1E0BB2E10E0E5010894A11CB11C1D157F
:1039A00018F40E94261C01C08FEF88831F5F17FF49
:1039B000F2CF38E7931609F0D4C0063409F03DC0C1
:1039C0008FEFE81687E3F80608F033C0CD2DA70186
:1039D00066277727440F551F661F771F6A017B01F3
:1039E000A2E0B1E011E08D9199272D913327322F7C
:1039F0002227822B932B0C01FA0110935700E89594
:103A000011244E5F5F4F6F4F7F4FC25061F785E0CB
:103A1000F60180935700E89507B600FCFDCF81E1E1
:103A200080935700E89576956795579547957A0165
:103A300089C080E00E941E1C85C0053409F082C048
:103A4000F7012D2DA2E0B1E0E1BD8F2F992782BDB6
:103A50008D9180BD3196FA9AF99AF999FECF21504D
:103A600099F77F016FC0873609F03DC00E94261C80
:103A70000E94261CC82F0E94261C863419F5C701F7
:103A8000AA27BB276C017D01CC0CDD1CEE1CFF1CA2
:103A9000F60105911491802F0E941E1C812F9927F9
:103AA0000E941E1C82E090E0A0E0B0E0C80ED91E8B
:103AB000EA1EFB1EC25061F7F694E794D794C794B0
:103AC000760139CF853409F036CFE1BC8F2D9927A7
:103AD00082BDF89A0894E11CF11C80B50E941E1C5E
:103AE000C15099F728CF853601F598E7991651F519
:103AF00080E090E0A0E0B0E023E0FC0120935700DC
:103B0000E89507B600FCFDCF80589F4FAF4FBF4FE1
:103B10008F3F37E3930730E0A30730E0B30768F344
:103B200081E180935700E8950DC0853469F488E100
:103B300090E02CE00FB6F894A895809360000FBE3B
:103B4000209360008DE030C08035E1F38C34D1F3F8
:103B5000803711F483E528C0843729F488E70E9470
:103B60001E1C80E021C0843521F40E94261C982E62
:103B7000E9CF8B3109F4DDCE8A3A09F4DACE863505
:103B800029F480E30E941E1C82E30EC0833741F4B7
:103B900086E00E941E1C84E90E941E1C8EE104C067
:0E3BA0008B3109F4C8CE8FE30E941E1CC4CEE8
:0400000300003800C1
:00000001FF
